:1000000000308A00EF2800008316051283120512C3
:10001000831685128312851200348316851283128B
:100020008516831605128312051200342F308400C2
:100030008313000803192D280130A100BF30A00050
:100040006400A00B2028A10B1E284A30A000A00BA2
:10005000272800006400800B1C280034A70104201E
:100060002708463C031C4728A70A270883169B003D
:100070009C131C141A088312A800A808031D422808
:100080000D20432804209630AF001620302800347D
:10009000AE012D082E0203185A284B30AF0016204F
:1000A0000D209630AF00162004204B30AF001620F4
:1000B000AE0A492800342810A708031D6428AB01A4
:1000C000AA014730A9007028DF30AB00AA01FF3039
:1000D000A9002A08003C031870280A30AD00482007
:1000E000831605108312051483160511831205115A
:1000F0000A30AF001620AA08031D822829082B0207
:100100000318A828003028180130AD000030191B52
:1001100001302D06AC00AB0A2B0883169B0083121E
:100120002C0883169A001C1583120B08A0008B1351
:10013000831655309D00AA309D009C149C189E2863
:100140001C11831220088B049630AF0016207B28E8
:1001500083160510831205108316051183120511ED
:10016000A708031DC82883169B0199309A001C1507
:1001700083120B08A0008B13831655309D00AA3004
:100180009D009C149C18C2281C11831220088B040B
:100190000034AA01E030A7002708A70AAB008316A5
:1001A0009B009C131C141A088312A900270FD9283E
:1001B000EB282708A70AAB0083169B009C131C148E
:1001C0001A088312A800290828020319EA28AA0A93
:1001D0002808A900D62803102A0CA1003929840177
:1001E00083131F308305613083168F0083121F1322
:1001F00083161F109F101F119F1107308312990043
:1002000083168501831285011F1383161F109F100B
:100210001F119F1183121F100430990083160508C7
:1002200002388500640002308312A000A00B16295A
:10023000192919088C11AF308316990061308F008D
:100240009B019C131C141A08993C031D2A29831234
:100250002E2083168312A601A608031D3C29023016
:10026000AD0048200130A7005B200230AD004820DF
:10027000C9282108A6002C292608013A0319472974
:10028000033A03194C29013A031951295329A701AB
:100290005B200230AD0048202E200230AD00482007
:0C02A00054292E20512963002B296300F3
:02400E00E43399
:00000001FF
